:100000008316133085000030860083128601850137
:1000100096018C019201930194018D018E018F0153
:10002000900191015B207C200C08AA3A031DD02886
:100030007F205B207C200C08003A031DD028F43080
:100040008C00B7207F20CC209C205B207C200C08DB
:10005000FA3A031DD028051E3229111019218617DE
:100060008D018E018F019001FF30980010309900B2
:100070007F2052207C200C088D0086177F205B207B
:100080007C200C088E007F205B207C200C088F00D9
:10009000111C4F287F205B207C200C089000E3205F
:1000A00086133028051C5D28980B5228990B52287E
:1000B00086010511851105185B28051C5D28722035
:1000C0007220722072207220722072207220051815
:1000D00067288518702812109720051C6D280800C5
:1000E00012146C280518722805089400940C940CBE
:1000F0008C0C051C792808008320CC20080083166E
:1001000005148312080083160510831205100800D9
:1001100083168510831285100800831685148312B8
:1001200008008C0C03189628882097288D20051C21
:1001300097280518992808007C20CE208820CE20FA
:100140007F200518A12891209120912091209120B5
:10015000912091209120B42097208D209720051C7C
:10016000AF28851CB128080012188D288828930113
:100170000C18930A8C18930A0C19930A8C19930A79
:100180000C1A930A8C1A930A0C1B930A8C1B930A61
:100190001210131C12140800950BCC280000080044
:1001A000FF309800FF3099008617980BD428990BE0
:1001B000D428FF309800FF3099008613980BDD2873
:1001C000990BDD28D02896010D1896168D18161754
:1001D0000D1916160D1AF1280E08FF39031D961574
:1001E000F8280E0897009709170AFF39031D1615FE
:1001F0008D1AFF280F08FF39031D161406290F0852
:1002000097009709170AFF39031D9614111C162928
:1002100090190F2910080739031D05151629100814
:1002200097009709170A0739031D851516088600D8
:100230000800E8308C00B7207F20CC209C205B2079
:100240007C200C08FA3A031DD02801308C00B7201E
:100250007F20CC209C205B207C200C08FA3A031DD8
:10026000D0280800F3308C00B7207F20CC209C20C1
:100270005B207C200C08FA3A031DD028C8308C0083
:10028000B7207F20CC209C205B207C200C08FA3AF1
:10029000031DD028F3308C00B7207F20CC209C2079
:1002A0005B207C200C08FA3A031DD02864308C00B7
:1002B000B7207F20CC209C205B207C200C08FA3AC1
:1002C000031DD028F3308C00B7207F20CC209C2049
:1002D0005B207C200C08FA3A031DD02850308C009B
:1002E000B7207F20CC209C205B207C200C08FA3A91
:1002F000031DD028F2308C00B7207F20CC209C201A
:100300005B207C200C08FA3A031DD0287F205B205C
:100310007C200C08033A031DD028111419218617DC
:02032000302883
:02400E00F13F80
:00000001FF
